:1000000039C051C050C04FC04EC04DC0C6C04BC01B
:100010004AC049C048C047C046C045C044C043C0AC
:1000200042C041C040C03FC03EC0000000000000D0
:1000300000020000000103040000000000003B007B
:1000400038000000320000003A00370000003100A4
:100050000404010104040404040202020202020274
:1000600002010102020104081020400102040810EC
:100070002040800411241FBECFEDCDBF10E0A0E6CC
:10008000B0E0EEE8F4E002C005900D92A637B107AB
:10009000D9F720E0A6E7B0E001C01D92A738B2076B
:1000A000E1F7C5D0F2C1ACCF90E0FC01EE59FF4FB3
:1000B0002491805B9F4FFC018491882399F090E00C
:1000C000880F991FFC01EA5BFF4FA591B491FC01D9
:1000D000E45CFF4F859194918FB7F894EC91E22BFB
:1000E000EC938FBF089590E0FC01E65DFF4F3491E3
:1000F000FC01EE59FF4F2491FC01E05BFF4FE491BE
:10010000EE23B9F0332329F03130A1F480B78F7793
:1001100080BFF0E0EE0FFF1FE45CFF4FA591B491AC
:100120008FB7611117C0F894EC9120952E232C9372
:100130008FBF0895323019F480B78F7DE9CF333007
:1001400021F48FB58F778FBDE4CF343011F78FB5A1
:100150008F7DF9CFF894EC912E2BE9CF0F931F935D
:10016000CF93DF93C7E0D0E0082F10E0B8010C2E4A
:1001700002C0759567950A94E2F7617084E0B3DF79
:1001800061E086E0B0DF60E086E0ADDF219770F7E8
:10019000DF91CF911F910F9108951F920F920FB68B
:1001A0000F9211242F933F938F939F93AF93BF93FD
:1001B00080917B0090917C00A0917D00B0917E00A9
:1001C00030917A0026E0230F2D3768F129E8230FBC
:1001D0000396A11DB11D20937A0080937B0090931C
:1001E0007C00A0937D00B0937E008091760090917A
:1001F0007700A0917800B09179000196A11DB11D02
:100200008093760090937700A0937800B093790064
:10021000BF91AF919F918F913F912F910F900FBE02
:100220000F901F9018950296A11DB11DD4CF83E0A9
:1002300080BF83BF789489B7826089BF85E034DF4F
:1002400086E032DF84E030DF8BE02EDF8AE02CDFD7
:1002500089E02ADF88E028DF60E08BE044DF60E0AF
:100260008AE041DF60E089E03EDF60E088E03BDF7C
:1002700088EEC82E83E0D82EE12CF12C92E7892E4F
:1002800099249394A12CB12C2CE3422E512C612C57
:10029000712C0AE02FB7F89460917B0070917C007C
:1002A00080917D0090917E002FBFA7019601CBD059
:1002B000223781E038074105510508F47DC01092CE
:1002C00083001092840010928500109286002FB750
:1002D000F89480917B0090917C00A0917D00B0917A
:1002E0007E002FBF40917F0050918000609181007F
:1002F00070918200841B950BA60BB70B853F914034
:10030000A105B105F0F0809161008530D0F481E065
:1003100090916000911180E0809360002FB7F89475
:1003200080917B0090917C00A0917D00B0917E0037
:100330002FBF80937F0090938000A0938100B093A3
:10034000820080916000813009F0A4CFC3E8D0E042
:1003500010E060E0123009F451C0133009F459C0C4
:10036000113009F440C08AE0BEDE60E089E0BBDE07
:1003700060E088E0B8DE61E08BE0B5DE399060E0F7
:1003800085E0B1DE832D90E0113009F04DC0845935
:100390009F4FFC0180818095E1DE61E085E0A3DE76
:1003A00060E085E0A0DE8FEFD9DE61E085E09BDED6
:1003B0001F5F143071F66ECFC501B401621B730B61
:1003C000840B950BA30192013ED0862F20936100F0
:1003D0001092830020938400602F29D080938500A1
:1003E0009093860074CF8BE07EDE60E089E07BDE58
:1003F00060E088E078DE61E08AE0BFCF8BE073DE0A
:1004000060E08AE070DE60E088E06DDE61E089E057
:10041000B4CF8BE068DE60E08AE065DE60E089E012
:1004200062DE61E088E0A9CF8E599F4FB2CF991B61
:1004300079E004C0991F961708F0961B881F7A95DB
:10044000C9F780950895A1E21A2EAA1BBB1BFD01D6
:100450000DC0AA1FBB1FEE1FFF1FA217B307E407A3
:10046000F50720F0A21BB30BE40BF50B661F771FFB
:10047000881F991F1A9469F76095709580959095DB
:0E0480009B01AC01BD01CF010895F894FFCFA0
:10048E000106FC60DAF266B6BEE0FEF6FD61DBF355
:06049E0067B7BFE1FFF7A4
:00000001FF
